:020000040000FA
:1000000083160313273085008601831203138601AC
:10001000FF309F008B010130A8000130A700203085
:10002000A300AA30A4004430A5007E30A900AA3065
:10003000AA000430AB00FF30AC00FF30AD000A3046
:10004000A600271C5A21851C2C20051C2E2094203C
:10005000C830850472202128A60A2F28A603260866
:10006000FF3A0319A60A2608F53E0318A60303184B
:1000700033288B13003083169B00831226088316C7
:100080009A001C1555309D00AA309D009C148312C7
:10009000C83085048C1F4A288C13A930A000453035
:1000A000A1000230A200A00B5328A10B5328A20BE1
:1000B00053280800C8308504851C6428051C642862
:1000C0000301813E86005C28000000000000AC0BAC
:1000D0006428AD0B64287E30A900AA30AA00043041
:1000E000AB000800051D7728051974287928051D1F
:1000F00077282908003A031D86282A08003A031D9C
:1001000086282B08003A031D86285A28A90B8B281D
:10011000AA0B8B28AB0308002808003A0319912882
:10012000A80BA528A701A5282308003A031D9F288E
:100130002408003A03192508003A03198C28A30B58
:10014000A528A40BA528A50B000026080A3A031928
:10015000D2282608003A0319D8282608013A03199C
:10016000DC282608023A0319EA282608033A03196C
:10017000F8282608043A031906292608053A03191F
:1001800014292608063A031922292608073A0319D2
:1001900030292608083A03193E292608093A031986
:1001A0004C290800373085050301253E86002128AB
:1001B0000301813E860008001530A0000A30A1002E
:1001C000A00BE028A10BE028373085050301ED3EA8
:1001D000860008006F30A0000930A100A00BEE28B7
:1001E000A10BEE28373085050301433E8600080049
:1001F000C930A0000830A100A00BFC28A10BFC28EE
:10020000373085050301493E860008002330A000F1
:100210000830A100A00B0A29A10B0A293730850557
:1002200003012D3E860008007D30A0000730A100AC
:10023000A00B1829A10B1829373085050301193E99
:1002400086000800D730A0000630A100A00B2629A8
:10025000A10B2629373085050301113E86000800D1
:100260003030A0000630A100A00B3429A10B3429A6
:10027000373085050301CD3E860008008A30A00096
:100280000530A100A00B4229A10B4229373085057A
:100290000301013E86000800E430A0000430A10004
:1002A000A00B5029A10B5029373085050301093EC9
:1002B000860008008316031300309B001C141A08E4
:0802C0008312A600A70A080042
:02400E00303F41
:00000001FF
